:100000000C9429030C947C030C947C030C947C03C7
:100010000C947C030C947C030C947C030C947C0364
:100020000C947C030C947C030C9464250C947C034A
:100030000C943B250C947C030C947C030C947C0363
:100040000C947C030C947C030C947C030C947C0334
:100050000C947C030C94422A0C947C030C947C0337
:100060000C947C030C947C030C947C030C947C0314
:100070000C947C030C947C030C947C030C947C0304
:100080000C947C030C947C030C947C030C947C03F4
:100090000C947C030C947C030C947C030C947C03E4
:1000A0000C947C030C947C030C947C030D0A676510
:1000B00074446576446573637220000D0A73657439
:1000C000436F6E6620000D0A00424D20636F6E661E
:1000D0006967757265640D0A000D0A005257553A3A
:1000E00020000D0A0052504950453A20000D0A00E8
:1000F0005345545F49444C453A20000D0A0053458E
:10010000545F50524F544F434F4C3A2000736B6929
:1001100070205345545F50524F544F434F4C0A0088
:100120000D0A000D0A496E746572666163653A00D6
:100130000D0A00624E756D49666163653A000D0AED
:10014000006249666163654E756D3A000D0A0043B1
:100150006E663A000D0A00624E756D45503A0048D1
:1001600049445F50524F544F434F4C5F4B455942A7
:100170004F4152440D0A000D0A004E433A000D0A49
:1001800000416464723A000D0A007365744164644E
:10019000723A006570696E666F0D0A00424D204923
:1001A0006E69740D0A000D0A0020000D0A0028680F
:1001B0006964626F6F742E682920496E7465726677
:1001C0006163653A000D0A0028686964626F6F74A4
:1001D0002E682920537472616E67652072656164B0
:1001E00020636F756E743A20000D0A0028686964F8
:1001F000626F6F742E682920506F6C6C3A000D0A84
:100200000028686964626F6F742E682920657049E0
:100210006E666F5B6570496E746572727570744955
:100220006E496E646578202B20695D2E6D61785073
:100230006B7453697A653D000D0A00286869646231
:100240006F6F742E6829206570496E666F5B6570EC
:10025000496E74657272757074496E496E64657822
:10026000202B20695D2E6570416464723D000D0A8B
:100270000028686964626F6F742E682920693D00E8
:10028000526F6C6C6F766572206572726F723A2075
:1002900069676E6F7265640D0A002069676E6F7220
:1002A00065640D0A000D0A00202530325800696E81
:1002B0007075742025643A003E3E3E3E48554252D9
:1002C00053540A003E3E3E3E4255535253540A0098
:1002D0003E3E4855425253540A003E3E4255535208
:1002E00053540A002E2E2E4641494C0D0A004275E9
:1002F0006666657220706F696E746572206973201E
:100300004E554C4C210D0A00733A25730A00753A7C
:10031000253032580A005B695D005B735D007370C5
:100320006565643A2025730A007573625F737461B2
:1003300074653A20253032580A00686F73742E5461
:1003400061736B3A2025640A004C45443A202530FD
:1003500032580A000A4C6F6F702073746172742EE9
:100360000A000A55534220636F6E666967757265AD
:10037000642E0A000A544D4B3A3836313537642F13
:100380004C5546413A6436613764662F55485332BE
:100390003A6466386536340A005B705D005B535D15
:1003A000005B505D005B575D000631FF0974A101E1
:1003B0000975150026FF009520750881020976153C
:1003C0000026FF00952075089102C005010906A1CD
:1003D00001050719E029E715002501950875018138
:1003E0000295017508810105081901290595057512
:1003F0000191029501750391010507190029FF1567
:100400000026FF00950675088100C009023B000226
:100410000100A032090400000103010100092111BB
:100420000100012240000705810308000A090401B8
:100430000001030000000921110100012222000730
:100440000583032000011201100100000008EDFEE9
:100450005B001508010200013C03550053004200F7
:10046000200074006F00200055005300420020005F
:100470006B006500790062006F006100720064002B
:10048000200063006F006E0076006500720074004B
:10049000650072000000080354004D004B0000008E
:1004A0000403090473797374656D3A202530345858
:1004B0000A00636F6E73756D65723A20253034588B
:1004C0000A00000000000405060708090A0B0C0DCD
:1004D0000E0F101112131415161718191A1B1C1DC4
:1004E0001E1F202122232425262728292A2B2C2DB4
:1004F0002E2F303132333435363738393A3B3C3DA4
:100500003E3F404142434445464748494A4B4C4D93
:100510004E4F505152535455565758595A5B5C5D83
:100520005E5F606162636465A56768696A6B6C6D34
:100530006E6F707172737475767778797A7B7C7D63
:100540007EA8A9AA00000085008788898A8B000000
:10055000000090910000000000000000000000007A
:10056000000000000000000000000000000000008B
:10057000000000000000000000000000000000007B
:10058000000000000000000000000000000000006B
:10059000000000000000000000000000000000005B
:1005A0000000E0E1E2E3E4E5E6E70000000000002F
:1005B000000000000000000000000000000000003B
:1005C00000000A002530325820006B6579626F61A7
:1005D00072643A20000D0A00285553423A3A496E97
:1005E0005472616E73666572292065702072657140
:1005F00075657374656420000D0A00285553423AEE
:100600003A496E5472616E73666572292061646442
:10061000722072657175657374656420000D0A003F
:10062000285553423A3A496E5472616E7366657248
:10063000292053657441646472657373204661694F
:100640006C656420000D0A004552524F523A00007A
:10065000492411241FBECFEFDAE0DEBFCDBF04B6C0
:1006600003FE28C08091900590919105A09192057C
:10067000B09193058730904BA740B04BD9F41092BE
:10068000900510929105109292051092930514BE58
:100690000FB6F894A89580916000886180936000FF
:1006A000109260000FBE1092010810920008E0E066
:1006B000F8E3099511E0A0E0B1E0E0E9F7E502C058
:1006C00005900D92AC38B107D9F725E0ACE8B1E060
:1006D00001C01D92A039B207E1F713E0C9E2D3E0EF
:1006E00004C02197FE010E94C02BC832D107C9F770
:1006F0000E94E4260C94C62B0C940000FF93EF9309
:10070000E0918C01F0918D01309709F00995EF91FE
:10071000FF910895FC018591803011F0EFDFFBCF50
:100720000895FF27E0E230E247FF0CC0419597FFB4
:1007300009C0EDE26095709580959095611D711DE1
:10074000811D911D27FF02C0219530E350E2AA27A9
:10075000660F771F881F991FAA1FA41710F0A41BEC
:1007600063955A95A9F7AA3008F0A95FA05DAF93E9
:10077000F395611571058105910541F7ED3211F48D
:10078000EF93F395F21718F43F93F395FBCF8F9106
:10079000B5DFFA95E1F70895E991F99185918030F7
:1007A00021F0853219F0AADFF9CF089520E0E8940E
:1007B00055915532C1F3503311F4689455915A3321
:1007C00048F4505390F3220F022E220F220F200DD7
:1007D000250FF4CF0EF4219589919991533619F391
:1007E000533729F1533559F1BC0188279927E894EB
:1007F0005C3621F48991999168945591543639F475
:1008000046EF7EF077FF0DC08FEF9FEF0AC05537A0
:100810004AE039F0583540E121F0523642E009F023
:100820000895FF93EF937DDFEF91FF91B7CFFF9393
:10083000EF93FC0181918030B9F360DFFBCFFF9330
:10084000EF9368DFF1CFDF93CF93CDB7DEB7259677
:10085000A3DFCF91DF910895FC0189E195E09583B5
:10086000848383E391E09183808381E591E09383A6
:100870008283108E118E128E138E148E168E81E04E
:10088000878B168A148A178288E080878CE3818799
:100890001286138684E08487158616868787108AD9
:1008A000118AAFE6B5E090E080E02D913D91232BD9
:1008B00041F4880F991FDC01A159BA4FED93FC93C5
:1008C000089501968031910581F70895EEE8F2E0F0
:1008D0009281891301C01282319692E0E439F907BE
:1008E000B9F70895A0E9B2E0EFEF90E02D918217FB
:1008F00051F0EF3F19F4211101C0E92F9F5F9630AD
:10090000A9F7EF3F09F408950E2E000CFF0BE257F4
:10091000FD4F82830895E091EA03F091EB03309755
:1009200021F00190F081E02D099480E00895E8ED38
:10093000F0E080818E7F80831092E2001092DA00D6
:100940001092E100A0EEB0E08C9181608C938081E8
:100950008F77808319BCA7EDB0E08C918E7F8C934C
:1009600080818F7E80831092CD0208950E9497042B
:10097000F89487E797E7909301088093000887E051
:1009800090EBDC018093900590939105A0939205E4
:10099000B093930588E19CE00FB6F894A8958093F6
:1009A00060000FBE90936000FFCFFC018091E202D7
:1009B0009091E30286179707A0F06115710529F45D
:1009C0009091E8009E779093E80090E061157105A2
:1009D00051F4911108C08091E80082FF35C080E099
:1009E0000895BC01F2CF8091E4028823C9F18530DB
:1009F000C9F18091E80083FD31C08091E80082FD5B
:100A0000EACF8091E80080FFE1CF2091F300809150
:100A1000F200322F282F6115710519F028303105A9
:100A200058F091E02830310509F090E02091E8007D
:100A30002E772093E800CACF81918093F100615016
:100A400071092F5F3F4FE7CF8091E402882341F087
:100A5000853041F08091E80083FFBDCF81E00895AB
:100A600082E0089583E008952091E4003091E5004C
:100A700085E69091EC0090FF06C09091E80090FF11
:100A800006C080E008959091E80092FDFACF909121
:100A9000E402992391F0953091F09091EB0095FD4F
:100AA00010C04091E4005091E5002417350709F388
:100AB00081509A01F1F684E0089582E0089583E080
:100AC000089581E008958091DC0287FF13C0809132
:100AD000E80082FF06C08091E8008B778093E800F1
:100AE00004C08091E4028111F2CF08958091E40264
:100AF0008823D9F38091E80080FFF8CF8091E80047
:100B00008E77ECCF982F9093E900242F762F50E02A
:100B1000891731F07091EC002091ED005091F000B8
:100B200021FD07C09F5F973071F78093E90081E056
:100B300008953091EB003E7F3093EB003091ED0053
:100B40003D7F3093ED003091EB0031603093EB004E
:100B50007093EC002093ED005093F0002091EE0094
:100B600027FDE0CF80E008950F931F93CF93DF938D
:100B7000CDB7DEB7AA970FB6F894DEBF0FBECDBFD4
:100B80008091E402882309F423C11091E9001F70C9
:100B90008091EC0080FF39C080E8182B1092E900AA
:100BA0008091E80083FF11C1ECEDF2E084EE92E069
:100BB0002091F10021938E179F07D1F78091DD02DC
:100BC000833009F470C018F5813009F447C08230D1
:100BD00009F4AFC08091E80083FFE9C08091DC0296
:100BE0009091DD029A3008F0E2C0E92FF0E0E55084
:100BF000FA4F0C94C02BAA06D006D706D006D7060B
:100C000032075407D70650085D0880E0C6CF8A3007
:100C100009F47EC08B3009F463C08930D9F6809125
:100C2000DC028132B9F68091E0029091E102892BD9
:100C300089F68091E800877F8093E8008091E80042
:100C400082FF2CC08091F1008093D0028091E80057
:100C50008B778093E8000E946305BCCF8091DC0213
:100C6000813A09F0B7CF8091E800877F8093E80050
:100C70008091E0029091E102892B61F060E090E0C8
:100C800080E070E00E94D5048091E8008B7780932B
:100C9000E800A0CF68E081ED92E0F3CF8091E4021C
:100CA0008111CCCF97CF8091DC02813A09F092CFAD
:100CB0008091E0029091E102892B09F08BCF809125
:100CC000E800877F8093E8008091E80080FFFCCFF8
:100CD000809110018093F1008091E8008E77B9CF68
:100CE0008091DC02813209F075CF8091E002909111
:100CF000E102892B09F06ECF8091E800877F809315
:100D0000E8000E9463058091DE028093100162CFAB
:100D10008091DC02813209F05DCF8091E800877F0D
:100D20008093E8000E9463058091DF028093CF02E8
:100D300051CF8091DC02813A09F04CCF8091E800DC
:100D4000877F8093E8008091E80080FFFCCF80914E
:100D5000CF02C0CF803889F0823849F58091E00217
:100D60008F70873020F58093E9008091EB0085FB40
:100D7000882780F91092E90006C08091D9029091ED
:100D8000DA02911182609091E800977F9093E800D9
:100D90008093F1001092F1008091E8008E7731C0CD
:100DA000282F2D7F21F48823F1F0823079F1809172
:100DB000E80083FF0AC08091E800877F8093E80005
:100DC0008091EB0080628093EB001F701093E9002C
:100DD000AA960FB6F894DEBF0FBECDBFDF91CF91BC
:100DE0001F910F9108958091DE02813001F79330B9
:100DF00009F080E08093DA021092E9008091E80027
:100E0000877F8093E8000E946305D1CF8091DE0246
:100E10008111F2CF8091E0028F702FEF280F2630E2
:100E200030F68093E9002091EB0020FFE5CF93306E
:100E300031F48091EB0080628093EB00DDCF9091E4
:100E4000EB0090619093EB0021E030E001C0220FB5
:100E50008A95EAF72093EA001092EA008091EB006D
:100E60008860EACF8111A3CF0091DE020F778091D5
:100E7000E3008078802B8093E3008091E800877FF7
:100E80008093E8000E9463058091E80080FFFCCF1A
:100E90008091E30080688093E30083E0011101C04A
:100EA00082E08093E40283CF8058823008F07FCFC5
:100EB0002091DE023091DF022C3D83E03807A1F55E
:100EC00083E08A838AE289834FB7F894DE01139620
:100ED00020E03EE051E2E32FF0E050935700E49130
:100EE00020FF03C0E295EF703F5FEF708E2F90E020
:100EF000EA30C0F0C7968D939D932F5F243159F748
:100F00004FBF8091E800877F8093E8006AE270E03D
:100F1000CE0101960E94D5048091E8008B778093E2
:100F2000E80045CFC096E7CF4091E0025091E10242
:100F3000832F99278330910509F440C070F58130E3
:100F4000910509F46BC0029709F031CF8BE390E073
:100F5000EBE0F4E02091E800277F2093E800209167
:100F6000E2023091E3028217930708F49C0140E00B
:100F70002115310509F061C041115FC08091E80081
:100F800082FDCACF8091E402882331F2853021F2BC
:100F90008091E80083FFF2CFBFCF8132910591F1BC
:100FA0008232910509F003CF4115510509F440C083
:100FB000E9EAF3E04130510569F2F9CE33272130F7
:100FC0003105C1F060F02230310509F0F0CEE8E5DE
:100FD000F4E0E4918E2F90E0E8E5F4E007C0E0EA69
:100FE000F4E0E4918E2F90E0E0EAF4E0009709F459
:100FF000DECEB0CFE6E9F4E0E4918E2F90E0E6E9B2
:10100000F4E0F4CF4115510571F089E090E0E6E39A
:10101000F4E04130510509F49DCFC9CE82E190E062
:10102000E6E4F4E097CF89E090E0EDE1F4E092CFE0
:1010300080E490E0EBECF3E08DCF8091E402882334
:1010400009F46ACF853009F467CF8091E80083FD09
:1010500063CF8091E80082FD91CF8091E80080FF0E
:1010600087CF8091F3009091F200892798278927F4
:101070002115310519F08830910550F041E00897AD
:1010800009F040E08091E8008E778093E80070CF0F
:1010900044914093F1003196215031090196E8CFF7
:1010A000803809F084CE8091E800877F8093E80043
:1010B0008091DB028093F1006FCE811178CE009198
:1010C000DE02023008F073CE8091E800877F8093C3
:1010D000E8000093DB020E946305002371F084E0C6
:1010E0008093E40242E061EC81E00E94820546E2E6
:1010F00061EC83E00E9482055ACE8091E30087FD77
:10110000EECF81E0EDCFCF92DF92EF92FF920F937F
:101110001F93CF93DF93C8EDD0E088818F7E8883C3
:10112000E7EDF0E080818160808384E082BF81E030
:101130008093CD0288818E7F888302EE10E0F801D3
:1011400010821092DA0081EEC82ED12CF6011082A6
:1011500088818F77888388818068888388818F7D64
:10116000888319BC1092E4021092DB021092DA021A
:101170001092D90290EEE92EF12CF70180818B7F3D
:10118000808388818160888342E060E080E00E9403
:101190008205F60180818E7F8083F80180818160E5
:1011A0008083808188608083F70180818E7F808347
:1011B000888180618883DF91CF911F910F91FF908B
:1011C000EF90DF90CF90089508950895089580914D
:1011D000D0020895CF93DF93EC018A819B81DC01DB
:1011E000ED91FC910480F581E02D6A8509958A8551
:1011F000813439F4EA81FB81EA58FF4F80818B7F8B
:1012000080831A861B861C861D861E861F86188A6A
:1012100080E0DF91CF91089581E0693009F080E0AE
:101220000895FC0182850895DF92EF92FF920F935B
:101230001F93CF93DF93EC0185E0E62EF12CFE01A6
:10124000869FE00DF11D1124908596FF24C0192F73
:10125000177001E085E0D82E8FEF800F8F3008F0F7
:1012600001E0602F70E0062FD69EF001D79EF00DB2
:101270001124EC0FFD1F80858695869586958770D5
:10128000181701F16F5F7F4F603168F38D81811313
:1012900002C011501D8385E08E9DF0018F9DF00DE1
:1012A0001124EC0FFD1F108681E0818712862296A3
:1012B000D783C683DF91CF911F910F91FF90EF905D
:1012C000DF900895CE010E941409C6CFFC0121E0F1
:1012D000613499F49C01255B3F4F61E0AC014E5FA6
:1012E0005F4F1586668717865487438735962E1776
:1012F0003F07B9F7FC01158208953585631729F07A
:101300002F5F35962031C9F70895622F0C94140988
:10131000CF93DF93FC0167FD12C0283080F4442393
:1013200019F08581873059F0EF01A1E0B0E08D859B
:10133000882349F111962596A031B105C1F780E0C7
:1013400018C085E08A9FE0018B9FD00D1124CE0F3D
:10135000DF1F442389F081E4888785818F5F85833F
:1013600025E02A9FC0012B9F900D1124E80FF91F43
:101370008085DF91CF91089581E08887F1CF277034
:10138000687B622B0FC06623E1F26770660F660F01
:10139000660F4423A1F3606485818F5F8583877026
:1013A000687F682B25E02A9FC0012B9F900D112498
:1013B000E80FF91F6087862FDCCFFC0121E0611167
:1013C00002C0069608953585631739F02F5F35966C
:1013D0002031C9F790E080E00895069635E0239F1C
:1013E000800D911D112408950F931F93CF93DF93C8
:1013F0002115310599F0E901042F162F0E94DD090E
:10140000FC0186ED309729F01283D183C0830383DA
:1014100080E0DF91CF911F910F91089588EDF9CF72
:1014200081E008952FB7F8946091EF037091F00375
:101430008091F1039091F2032FBF0895CF93C09153
:101440009702C1110BC00E94120A643C79408105C9
:10145000910520F081E080939702C1E08C2FCF911D
:1014600008952FB7F8948091EF039091F003A09125
:10147000F103B091F2032FBF0895EF92FF920F9303
:101480001F93CF93DF93D82F0FB607FE46C08091EE
:10149000E402843079F08091030190E0019620917C
:1014A000050130E0822393232091040128171906B7
:1014B00009F0D0C00E941E0A81110FC08091030163
:1014C00090E001962091050130E082239323209142
:1014D00004012817190609F0BDC00E94310A8C01C9
:1014E000C091E900CF708091EC0080FD38C080E0B1
:1014F000C82B83E08093E90085E0E82E8091EB0023
:1015000085FD08C08091EB0080FF04C08091EE0053
:1015100087FD45C0CF70C093E900E09103018E2F95
:1015200090E001962091050130E0822393232091E1
:1015300004012817190609F460C0809101019091F7
:101540000201E80FF92FF11DD083809103018F5F15
:101550009091050189238093030181E074C080E8A4
:10156000C7CFE0910101F0910201E80FF11D9081D8
:101570008F5F209105018223809304019093F100F5
:101580008091E80085FD0BC08091E80080FF07C0D6
:101590008091E8008E778093E800E09200018091CE
:1015A000040190910301981751F19091E80095FD85
:1015B000D8CF80E02BC01092F10034C0809103019D
:1015C00090E001962091050130E082239323209141
:1015D00004012817190609F09DCFF0900001FF20A3
:1015E00009F498CF0E94310A8017910709F486CF39
:1015F000FA94F09200018C0181CF80E024C08091A8
:10160000E80085FFD6CFD093F10081E02091F30070
:101610009091F200322F292F232B79F09091E8003E
:1016200090FF0BC09091E80095FDC5CF9091E80028
:101630009E779093E800E0920001882309F4BECFE2
:10164000CF70C093E900DF91CF911F910F91FF9070
:10165000EF900895E091030170CF0E943D0A80E071
:1016600008956138710511F00C943D0A0895CF93E7
:10167000DF936138710569F0009759F0EC01FE01C4
:1016800084912196882329F060E870E00E94310B54
:10169000F6CFDF91CF9108950F931F93CF93DF93F0
:1016A000FC018B01EA0180819181892B61F460E862
:1016B00070E08EEE92E00E94370B80E0DF91CF91D8
:1016C0001F910F9108959281992319F128813981F1
:1016D000232B99F3D8012D913C91D9014C91838111
:1016E000682F691B770B80819181860F971FDC0122
:1016F0004C9382818150828388819981019799835B
:101700008883D8018D919C91119701968D939C931C
:10171000DACF8381828381E0D1CF8F929F92AF9283
:10172000BF92CF92DF92EF92FF920E949C2A4B01D0
:101730005C0120E030E04AE755E40E942B2B6B016E
:101740007C0120E030E040E85FE30E94682A87FDEA
:1017500030C020E03FEF4FE757E4C701B6010E94D9
:10176000262B1816F4F420E030E040E251E4C501E5
:10177000B4010E942B2B0E946D2A20E931E06115F3
:10178000710549F4FF90EF90DF90CF90BF90AF903C
:101790009F908F900895C9010197F1F761507109E9
:1017A000EECFC701B6010E946D2ACB010197F1F778
:1017B000E9CF61E070E0F9CFEF92FF920F931F93B2
:1017C000CF93DF938A01EB017B01E40EF51ECE156A
:1017D000DF0521F089910E943D0AF9CFC801DF9110
:1017E000CF911F910F91FF90EF900895862F0E9447
:1017F0003D0A81E090E00895089581E090E0089529
:101800008FEF9FEF089590E080E008950895EF92A4
:10181000FF920F931F93CF93DF937C018B01CCE05A
:10182000D0E0C7010C2E02C0959587950A94E2F787
:10183000B801805D0E94310B2497CC3F8FEFD80711
:1018400081F7DF91CF911F910F91FF90EF90089555
:101850000F931F93CF93C82F8B01282F30E084E084
:10186000359527958A95E1F780E3820F8A3310F04A
:1018700087E3820FB8010E94310BCF7080E38C0F99
:101880008A3310F087E38C0FB801CF911F910F912D
:101890000C94310BEF92FF92CF93DF93FC01E701A1
:1018A0008789823028F0948996132CC0823051F5B4
:1018B000648B458B9B819370933021F59A8197FFC0
:1018C00021C09E81258D291708F4958F282F30E09F
:1018D000D901AA0FBB1FA20FB31FAE0FBF1F9A8162
:1018E0009F7017969C9317979C8118969C931897B6
:1018F00094E019969C932E0F3F1FD90151964C935B
:101900008F5F878BDF91CF91FF90EF900895EF92DB
:10191000FF920F9302970E944A0C0F91FF90EF9055
:10192000089570E0685F7F4F660F771F860F971FDF
:10193000FC0180819181089581E0613009F080E0AF
:10194000089581E0633009F080E00895FC0186810C
:101950000895CF93DF93EC018C819D81DC01ED91A3
:10196000FC910480F581E02D6E8109951C8A1D8A09
:1019700081E08F8B1E82188E198E1A8E1B8E1C8E04
:1019800080E0DF91CF9108952E9808952E9A0895C2
:101990000F931F93CF93DF93D82FC62F8A010E94F6
:1019A000C40CD260DEBDF8018C2F882339F00DB451
:1019B00007FEFDCF91919EBD8150F7CFC00FD12F73
:1019C000D11D0DB407FEFDCF0E94C60CCE01DF91E4
:1019D000CF911F910F910895CF93DF93C82FD62FEA
:1019E0000E94C40CC260CEBD0DB407FEFDCFDEBDAB
:1019F0000DB407FEFDCFDF91CF910C94C60CCF93B1
:101A0000C82F0E94C40CCEBD0DB407FEFDCF1EBC76
:101A10000DB407FEFDCF0E94C60C8EB5CF91089580
:101A20008F929F92AF92BF92CF92DF92EF92FF92EE
:101A30000F931F93CF93DF93882E962E5A010E9407
:101A4000120A6B017C0128E8C20E23E1D21EE11CC0
:101A5000F11CC0E010E000E0D0E098280E94120ADB
:101A60006C197D098E099F0997FF1EC0692D80EFB3
:101A70000E94EC0C0E94120A6C197D098E099F09C4
:101A800097FF09C088EC0E94FF0C87FFF3CF60E846
:101A900088EC0E94EC0C88EF0E94FF0CC82FCF70DE
:101AA000C43081F0CE30B9F08C2FDF91CF911F91EF
:101AB0000F91FF90EF90DF90CF90BF90AF909F90ED
:101AC0008F9008950F5F1F4FA114B10439F20A15CA
:101AD0001B0521F6E9CFDF5FD33009F0BFCFE4CF9C
:101AE000AF92BF92CF92DF92EF92FF920F931F932C
:101AF000CF93DF93EC01B62EA42E69010E94DD097D
:101B00007C0186EDE114F10409F447C0D701ED91A1
:101B1000FC91119787ED309709F43FC013969C9183
:101B200080E0981731F02081A21629F033968F5F5C
:101B3000F8CFF0E0E0E0D601ED93FC938BED309729
:101B400061F1228126952695203108F02FE081E071
:101B500090E0A0E0B0E004C0880F991FAA1FBB1F4F
:101B60002A95D2F70197F801918380836B2D80EE3F
:101B70000E94EC0C88ED0E94FF0CD70114969C91FA
:101B8000682F697F992329F0CA58DF4F6881626006
:101B9000682B88ED0E94EC0C80E0DF91CF911F91C3
:101BA0000F91FF90EF90DF90CF90BF90AF9008958E
:101BB0009F92AF92BF92CF92DF92EF92FF920F93DC
:101BC0001F93CF93DF936C01C42FD22F992493944A
:101BD000E62EF12CEE0CFF1CE80EF91E86E5E80E51
:101BE000F11CA42EB12CABE2AA0EB11CAA0CBB1C9A
:101BF000AC0CBD1CF70180819181DC01ED91FC9161
:101C00000280F381E02D202F4D2F6C2F0995182F86
:101C1000803E09F077C060E870E0C11163C08AEDD2
:101C200092E00E94370B61E088EE0E94EC0C88EE97
:101C30000E94FF0C80FDFBCF60E488EC0E94EC0C5E
:101C400088ED0E94FF0C682F686088ED0E94EC0C04
:101C500088EC0E94FF0C86FFFBCF66E670E080E018
:101C600090E00E948D0BF70180819181DC01ED9164
:101C7000FC910190F081E02D202F4D2F6C2F0995C4
:101C8000182F8D3009F05CC08FEF890D833008F478
:101C90003FC060E870E0C11156C084EC92E00E9441
:101CA000370B61E088EE0E94EC0C88EE0E94FF0C7E
:101CB00080FDFBCF60E488EC0E94EC0C88ED0E9474
:101CC000FF0C682F686088ED0E94EC0C88EC0E9485
:101CD000FF0C86FFFBCF66E670E080E090E00E949C
:101CE0008D0B21C080ED92E00E94370BF5018081C1
:101CF0009181DC01ED91FC910284F385E02D6D2F43
:101D00000995B1CF8D3061F48FEF890D833058F490
:101D100064E670E080E090E00E948D0B93946ACFBF
:101D2000882309F4A0CF812FDF91CF911F910F91CC
:101D3000FF90EF90DF90CF90BF90AF909F9008956D
:101D4000882389F3A6CF88EB92E00E94370B8C2F73
:101D500090E08B96880F991F8C0D9D1DFC01808152
:101D60009181DC01ED91FC910284F385E02D6D2FD2
:101D70000995D9CF88EC0E94FF0C85FF14C060E262
:101D800088EC0E94EC0C88EF0E94FF0C807C909104
:101D900011018917E1F180931101803409F150F4A8
:101DA000882379F108958091F903811130C064E0AE
:101DB00088EEE7CF803819F0803C09F1089588ED6E
:101DC0000E94FF0C9091F90381FD11C09230F9F04F
:101DD00061EC88ED0E94EC0C82E08093F903089599
:101DE00088ED0E94FF0C9091F90381FDEFCF9330B5
:101DF00071F063EC88ED0E94EC0C83E0EECF81E0A3
:101E0000ECCF61EC88ED0E94EC0C1092F903089580
:101E1000FC01848D089570E0685F7F4F660F771F27
:101E2000860F971FFC015183408381E00895CF9373
:101E3000DF93CDB7DEB728970FB6F894DEBF0FBE9D
:101E4000CDBFE22F29833A834B835C836D837E83EE
:101E50008F8398872091A2022E2B2093A202FE014D
:101E60003396AE01475F5F4F2191243060F0A4EAC2
:101E7000B2E090E080E03D91311111C08E559D4F50
:101E8000DC0112962C93E417F50771F728960FB62C
:101E9000F894DEBF0FBECDBFDF91CF9108950196BC
:101EA0008630910541F7EFCFCF93DF93FC01DA0144
:101EB0008281882359F0813069F081E02381348167
:101EC000232B09F080E0DF91CF91089534832383A1
:101ED00081E08283838194810097B1F02D913C91C0
:101EE0001197232B51F3019794838383EB0188810E
:101EF00099810196998388838D919C91119701977F
:101F000011969C938E93E6CF1282D7CF2F923F9259
:101F10004F925F926F927F928F929F92AF92BF92F9
:101F2000CF92DF92EF92FF920F931F93CF93DF93A5
:101F300000D000D0CDB7DEB76C017A8369835C83B3
:101F40004B832C0182E1480E511C83E0282E560160
:101F5000A7E0AA0EB11C12E0332433944601B0E18D
:101F60008B0E911C3601EBE06E0E711C29813A81BB
:101F70002115310509F4D4C0D60190968C91823098
:101F8000F1F0B0F5882309F45AC0813089F7AE0129
:101F90004F5F5F4FBE016D5F7F4FC5010E944C0BCD
:101FA000882309F4BDC0D6011596ED91FC911697D2
:101FB000808191968C939197818192968C93F60172
:101FC0005682458220A2D60192968C9192978430B7
:101FD00011F493961C92F60181A18250848325818D
:101FE0003681308727838287818784E080A305C07C
:101FF000833049F3843009F0BBCFD60192968C919F
:10200000843039F1853009F44FC0823009F079C04D
:10201000AE014F5F5F4FBE016D5F7F4FC5010E94F4
:102020004C0B882309F47CC0F601858984A3D60172
:1020300016969C928E92159790961C9297CFF601C9
:10204000148385819681908787831287118730A2B8
:102050009ECFAE014F5F5F4FBE016D5F7F4FC501E9
:102060000E944C0B882309F45BC0D60155968C91D5
:1020700055978330E1F656968C9156978130B9F694
:1020800098969C91989757968C91992351F0882314
:1020900071F2F60133A2928996A3938997A385A33F
:1020A000C6CF813021F6F5CFAE014F5F5F4FBE0145
:1020B0006D5F7F4FC5010E944C0B882389F1D601CB
:1020C00093968C919397882309F4B1CF12968D91B2
:1020D0009C91009709F4ABCFDC01ED91FC9101904C
:1020E000F081E02D7401D60195960C919597979605
:1020F0002C91979796964C91969794966C910995FA
:1021000096CFF60121A12250330BAE014F5F5F4FF6
:10211000BE016D5F7F4FC3010E94540F811187CFB5
:102120000F900F900F900F90DF91CF911F910F9113
:10213000FF90EF90DF90CF90BF90AF909F908F90E7
:102140007F906F905F904F903F902F9008952F92C7
:102150003F924F925F926F927F928F929F92AF9237
:10216000BF92CF92DF92EF92FF920F931F93CF9384
:10217000DF9300D000D0CDB7DEB76C017A836983DE
:102180005C834B832C0182E1480E511C83E0282E96
:102190005601A7E0AA0EB11C12E033243394460185
:1021A000B0E18B0E911C3601EBE06E0E711C2981A3
:1021B0003A812115310509F4CFC0D60190968C9152
:1021C0008230F1F0B0F5882309F45AC0813089F7E4
:1021D000AE014F5F5F4FBE016D5F7F4FC5010E9433
:1021E0004C0B882309F4B8C0D6011596ED91FC91EB
:1021F0001697808191968C939197818192968C937A
:10220000F6015682458220A2D60192968C91929731
:10221000843011F493961C92F60181A1825084833C
:1022200025813681308727838287818784E080A358
:1022300005C0833049F3843009F0BBCFD6019296B4
:102240008C91843039F1853009F44AC0823009F02C
:1022500074C0AE014F5F5F4FBE016D5F7F4FC50120
:102260000E944C0B882309F477C0F601858984A36A
:10227000D60116969C928E92159790961C9297CFA7
:10228000F601148385819681908787831287118751
:1022900030A29ECFAE014F5F5F4FBE016D5F7F4F9B
:1022A000C5010E944C0B882309F456C0D6015596EF
:1022B0008C9155978330E1F698969C919897579614
:1022C0008C91992351F0882399F2F60133A29289D7
:1022D00096A3938997A385A3CBCF813049F6F5CFF9
:1022E000AE014F5F5F4FBE016D5F7F4FC5010E9422
:1022F0004C0B882389F1D60193968C919397882370
:1023000009F4B6CF12968D919C91009709F4B0CF45
:10231000DC01ED91FC910190F081E02D7401D6017A
:1023200095960C91959797962C91979796964C9198
:10233000969794966C9109959BCFF60121A1225016
:10234000330BAE014F5F5F4FBE016D5F7F4FC30127
:102350000E94540F81118CCF0F900F900F900F900F
:10236000DF91CF911F910F91FF90EF90DF90CF9071
:10237000BF90AF909F908F907F906F905F904F90A5
:102380003F902F90089580E00895089580E008958B
:102390002F923F924F925F926F927F928F929F9275
:1023A000AF92BF92CF92DF92EF92FF920F931F9363
:1023B000CF93DF937B014A016901F901A080B180CD
:1023C000FB012180F90111821082FB01828160E111
:1023D00081FD60E288EE0E94EC0C3A2CA401F7012A
:1023E000608180E00E94100D582EF6E08F17B1F347
:1023F00081114EC088EC0E94FF0C82FF5DC080E31B
:102400000E94FF0C482E8A151B0411F008F0432C83
:10241000F601808191813501681A790A77FE02C040
:10242000712C612CC42DD0E0C615D7050CF43E01EB
:10243000562C0E94C40CF8E0FEBD0DB407FEFDCF83
:10244000F801552041F01EBC5A940DB407FEFDCF93
:102450008EB58193F6CF060D171D0E94C60C64E061
:1024600088EC0E94EC0CF60180819181C80FD91F85
:10247000D183C083421420F0CA15DB0508F4AECF27
:1024800088EF0E94FF0CF701928184FB91F99283FF
:10249000852DDF91CF911F910F91FF90EF90DF90ED
:1024A000CF90BF90AF909F908F907F906F905F90F4
:1024B0004F903F902F90089580EF582EE9CF2F92A4
:1024C0003F924F925F926F927F928F929F92AF92C4
:1024D000BF92CF92DF92EF92FF920F931F93CF9311
:1024E000DF93CDB7DEB765970FB6F894DEBF0FBEAA
:1024F000CDBF3C01342E222E402EED8AEAA4FBA44F
:10250000188A1F861E861D868E01035F1F4F9E013F
:10251000215F3F4F40E00E94700D582E81111AC17B
:1025200039822A824B822D892C83DE82CD82B88625
:10253000AF82AE014F5F5F4F68E080E20E94C80C3F
:102540004D855E8560E080E10E94100D811120C103
:10255000E114F10409F449C00F851889D8011296D5
:102560008C91129737FE47C0826012968C9365015A
:10257000C114D10409F411C19C2D8D2D8C149D041E
:1025800010F4982D892D9B878C874D855E856F85EE
:10259000788987019E01255F3F4FC3010E94C811C2
:1025A000582EB6E08B1721F38111D4C0ECA5FDA500
:1025B0003097A1F06B857C850190F081E02D019032
:1025C000F081E02DC5018C199D099A8789879E01AC
:1025D000275F3F4FA7018CA59DA509958B859C85FD
:1025E000C81AD90A8815990518F64D855E8537FEF3
:1025F000CBC080EACAC0816012968C931297119664
:102600006C908FEF860D803408F0C4C02D843E841A
:102610000E94120A9B01AC0128573C4E4F4F5F4F5E
:10262000298B3A8B4B8B5C8BD80112968C9160E88E
:1026300080FF60E488EE0E94EC0C512C712C811418
:10264000910409F476C063018614970408F46401C8
:10265000CD8AA7016C2D80E10E94C80C6C2D88E307
:102660000E94EC0CF8016081606280EF0E94EC0C2B
:1026700088EC0E94FF0C87FFFBCF60E888EC0E948B
:10268000EC0C88EF0E94FF0C8F70582E412CB12C5F
:10269000A12C552019F10E94120A29893A894B89E7
:1026A0005C89621B730B840B950B97FF17C036E098
:1026B0005316E9F04EE05416B1F054E0551209C03B
:1026C0008FEFA81AB80A2114310489F02A143B04A8
:1026D00071F460E088E30E94EC0C2DC08C189D081A
:1026E000EC0CFD1CACCF439493E0491691F360E0F1
:1026F00088E30E94EC0CD7016C9180E10E94EC0C05
:102700006D8988E30E94EC0CF8016081606280EFC3
:102710000E94EC0C88EC0E94FF0C87FFFBCF60E866
:1027200088EC0E94EC0C88EF0E94FF0C8F70582EF2
:10273000B0CF5110CECF88EF0E94FF0CD801129677
:102740009C91129785FB90F912969C934D855E851E
:102750005520D1F0852D65960FB6F894DEBF0FBEDB
:10276000CDBFDF91CF911F910F91FF90EF90DF9040
:10277000CF90BF90AF909F908F907F906F905F9021
:102780004F903F902F90089580E860E00E94100DD8
:10279000582EE0CF8AED582EDDCF4D855E85552031
:1027A00009F427CFD7CF8F929F92AF92BF92CF924B
:1027B000DF92EF920F93CF931F921F921F921F925F
:1027C000912C812CB12CA12CD12CC12CE12C062FC9
:1027D00025E040E060E00E945F12C82F6CE271E0EB
:1027E00080E090E00E948D0B0F900F900F900F9063
:1027F0008C2FCF910F91EF90DF90CF90BF90AF9043
:102800009F908F9008958F929F92AF92BF92CF9298
:10281000DF92EF920F931F921F923F932F934A01E3
:102820005A01D12CC12CEE24E39400E026E040E8CC
:102830000E945F120F900F900F900F900F91EF90EA
:10284000DF90CF90BF90AF909F908F9008958F9220
:102850009F92AF92BF92CF92DF92EF920F931F930E
:102860001F921F921F930F934A015A01D12CC12C22
:1028700032E0E32E022F26E040E80E945F120F9024
:102880000F900F900F901F910F91EF90DF90CF90CE
:10289000BF90AF909F908F9008955F926F927F92BC
:1028A0008F929F92AF92BF92CF92DF92EF92FF9260
:1028B0000F931F93CF93DF93CDB7DEB7C054D109E9
:1028C0000FB6F894DEBF0FBECDBF3C01F62E542EDE
:1028D000E22E932ECE0101966C018C01242F49E04B
:1028E00050E0C3010E942714811118C0AB80BC8046
:1028F0009F92EF92DF92CF9280E4882E912CD12C80
:10290000C12C92E0E92E052D26E040E86F2DC30191
:102910000E945F120F900F900F900F90C05CDF4FDE
:102920000FB6F894DEBF0FBECDBFDF91CF911F91E0
:102930000F91FF90EF90DF90CF90BF90AF909F905E
:102940008F907F906F905F9008958F929F92AF923B
:10295000BF92CF92DF92EF920F93C42ED12C1F9291
:102960001F921F921F92912C812CB12CA12CE12C33
:10297000062F21E043E2FC016285828193810E945F
:102980005F120F900F900F900F900F91EF90DF90CC
:10299000CF90BF90AF909F908F9008958F929F920D
:1029A000AF92BF92CF92DF92EF920F93C62ED12CAF
:1029B0001F921F925F934F9324E0822E912C34E05C
:1029C000A32EB12CE12C00E020E043EAFC0162855B
:1029D000828193810E945F120F900F900F900F9051
:1029E0000F91EF90DF90CF90BF90AF909F908F901E
:1029F00008958F929F92AF92BF92CF92DF92EF9203
:102A00000F93C42ED12C1F921F921F921F92912CB4
:102A1000812CB12CA12CE12C062F23E043E2FC01F8
:102A20006285828193810E945F120F900F900F90B8
:102A30000F900F91EF90DF90CF90BF90AF909F904D
:102A40008F900895CF92DF92FF920F931F93CF93B1
:102A5000DF9300D000D0CDB7DEB78C01F62E1982FF
:102A60001A821B821C82462F61E10E94A5144F2D01
:102A700060E1C8010E94A5144F2D64E0C8010E94C6
:102A8000F91483E0C82ED12CAE014F5F5F4F6F2D3C
:102A9000C8010E94CE14811114C089819A81AB8132
:102AA000BC819D7F83309140A041B10551F064E627
:102AB00070E080E090E00E948D0B81E0C81AD108A0
:102AC00019F74F2D64E1C8010E94A5144F2D60E154
:102AD000C8010E94A51464E170E080E090E00E94CB
:102AE0008D0B0F900F900F900F90DF91CF911F9152
:102AF0000F91FF90DF90CF9008952F923F924F92C9
:102B00005F926F927F928F929F92AF92BF92CF927D
:102B1000DF92EF92FF920F931F93CF93DF93CDB786
:102B2000DEB7E8970FB6F894DEBF0FBECDBFDC016D
:102B30001A963C9131112CC1922E242E362E3C0136
:102B4000FC01E280F380D701ED91FC910190F081CE
:102B5000E02D60E0C70109958C01009709F41BC1C5
:102B6000FC01C080D180C114D10409F417C1530104
:102B7000F4E0AF0EB11CDC011196BC92AE9214963B
:102B80009C92FE0131962F019F0148E050E060E0E9
:102B9000D30112968D919C910E940314982EF801F6
:102BA0001482811101C18D8191ED992E893059F5E1
:102BB0008980D701ED91FC910280F381E02D222DD7
:102BC00041E0632DC7010995F3018287882309F449
:102BD000E8C098859583682F828193810E94D313E2
:102BE000982ED801CD92DC92882339F1D701ED914E
:102BF000FC910480F581E02DD3011A966C91C701F8
:102C00000995F3011286892DE8960FB6F894DEBF78
:102C10000FBECDBFDF91CF911F910F91FF90EF902D
:102C2000DF90CF90BF90AF909F908F907F906F90EC
:102C30005F904F903F902F900895811082C0950132
:102C400042E0F3016285828193810E94F409982E0B
:102C500081118AC01F921F925F924F9258E0852E79
:102C6000912C68E0A62EB12CD12CC12C79E2E72E54
:102C700000E026E040EAF3016285828193810E94B0
:102C80005F12982E0F900F900F900F9081116CC0D3
:102C90008B81D3011B968C931B97820120E048E027
:102CA00050E01A966C911A9712968D919C910E9401
:102CB0002714982E811158C04B815C8120E0F301CC
:102CC0006285828193810E942714982E81114CC0C5
:102CD000498150E08E010F5D1F4F20E0D3011A960D
:102CE0006C911A9712968D919C910E942714982EA0
:102CF00081113AC01F921F921F921F92912C812C1A
:102D0000B12CA12CE12C0E8129E040E0F301628579
:102D1000828193810E945F12982E0F900F900F90E6
:102D20000F90811121C011E0D3011B968C911B974C
:102D3000811708F1412F68E0C3010E94F9141F5F59
:102D4000F3CF482D413208F040E250E09201D30128
:102D50001A966C911A9712968D919C910E94031469
:102D6000982E882309F46BCF60E870E084EE92E03F
:102D70000E94370B48CF1296ED91FC911397EA58B9
:102D8000FF4F80818460808381E050968C933BCF9D
:102D900049ED942E38CF36ED932E35CF27ED922E78
:102DA00032CF84ED982E2FCFD182C0822CCF2F929C
:102DB0003F924F925F926F927F928F929F92AF92CB
:102DC000BF92CF92DF92EF92FF920F931F93CF9318
:102DD000DF93CDB7DEB7CC57D1090FB6F894DEBF7D
:102DE0000FBECDBF3C01162F842E922EDC0114960F
:102DF000CD90DC9060E870E08CE991E00E94370BA8
:102E0000F301868181112AC3158ED601ED91FC91C3
:102E10000190F081E02D60E0C60109957C010097EA
:102E2000E1F416ED812FC458DF4F0FB6F894DEBFE2
:102E30000FBECDBFDF91CF911F910F91FF90EF900B
:102E4000DF90CF90BF90AF909F908F907F906F90CA
:102E50005F904F903F902F900895FC01A080B1802B
:102E6000A114B10441F460E870E083E991E00E94AC
:102E7000370B17EDD7CF2301F7E04F0E511CDC01C4
:102E800011965C924E9214969C929E0126593F4F49
:102E900048E050E060E0F301848195810E940314D2
:102EA000082F8111DDC2AB960FADAB97D701AD9264
:102EB000BC92D601ED91FC910280F381E02D282D8A
:102EC00040E0612FC6010995F301868314ED882344
:102ED00009F4A8CFE2969FADE2979087682F84818E
:102EE00095810E94D313182F882311F1D7011496CE
:102EF0001C92D601ED91FC910480F581E02DD30167
:102F000016966C91C6010995F301168260E870E08F
:102F10008AE891E00E94370B60E870E0812F0E9400
:102F2000280C60E870E087E891E00E94370B7ACFC8
:102F300060E870E081E891E00E94370B60E870E0A3
:102F4000D30116968C910E94280C60E870E08EE701
:102F500091E00E94370BF7011482D601ED91FC91AC
:102F60000190F081E02DD30116966C91C601099570
:102F7000009709F456CFFC019482920141E0D301FD
:102F800016966C91169714968D919C910E94F40957
:102F900001119DC0EC960FADEC9760E870E08AE7F8
:102FA00091E00E94370B60E870E0802F0E94280CAF
:102FB00060E870E087E791E00E94370B60E870E01E
:102FC0008FE591E00E94370B6301B2E0CB0ED11C7C
:102FD00031E2832E31E0932E41E4242E312C2C0E4D
:102FE0003D1EE0E12E0E311C57E2A52E51E0B52E1C
:102FF0007E01F1E1EF0EF11C011709F4A7C1239640
:103000009FAE8EAE23972596DFAECEAE2597269641
:103010001FAE26972B961FAE2B972C961FAE2C9784
:103020002F961FAE2F9761961FAE1EAE6197A29688
:103030001FAEA297A3961FAEA397A4961FAEA49708
:10304000AA961FAEAA9728963FAE2EAE28972A962C
:103050003FAE2EAE2A972E963FAE2EAE2E979E01F5
:103060002F5B3F4F412FF3016681848195810E9440
:103070004D14D30157968C915797823008F043C076
:10308000BA82A982DC82CB821D821A861B861E86AA
:10309000188A1F8619A21AA21BA219A6FF82EE8205
:1030A000F986E886FD86EC869E012F5F3F4F412F13
:1030B00016966C91169714968D919C910E944D14C2
:1030C000F3018789823008F03DC11F5F95CF03313E
:1030D00008F002E1402F50E09E0126593F4FD301F6
:1030E00016966C91169714968D919C910E940314DC
:1030F000082F882309F44ECF60E870E08CEA90E056
:103100000E94370B5AC1F1E0ED96FFAFED9760E8F2
:1031100070E087E591E00E94370B60E870E0D30132
:1031200057968C910E94280C60E870E084E591E04D
:103130000E94370BF301478911ED423008F43EC17C
:1031400092016681848195810E94F40960E870E0B3
:103150008FE491E00E94370B60E870E0D301549651
:103160008C910E94280C60E870E08CE491E00E9451
:10317000370B68EE73E080E090E00E948D0B1F92A9
:103180001F921F921F92912C812CB12CA12CD12C1B
:10319000C12CE12CF301048929E040E0668184819F
:1031A00095810E945F12182F0F900F900F900F9033
:1031B00081114DC168EE73E080E090E00E948D0BBC
:1031C00060E870E081E491E00E94370B60E870E015
:1031D000D30155968C910E94280C60E870E08EE334
:1031E00091E00E94370B60E870E083E391E00E9479
:1031F000370B60E870E0F30186890E94280C60E8D4
:1032000070E080E391E00E94370BF12C1E01F1E4A5
:103210002F0E311C4F2C512CD30157968C9181507D
:10322000990B481659060CF0DDC060E870E083E2A7
:1032300091E00E94370B460C571C60E870E0F201E9
:1032400082890E94280C60E870E080E291E00E9490
:10325000370BED96FFADED97F1117DC060E870E0A2
:103260008DE091E00E94370BD2015296CC90D12C88
:103270001F921F921F921F92912C812CB12CA12C76
:10328000E12C00E02AE041E2F3016681848195812E
:103290000E945F12082F60E870E080EF90E00E94CB
:1032A000370B60E870E0802F0E94280C60E870E027
:1032B0008DEE90E00E94370B0F900F900F900F90C3
:1032C000002319F0053009F078C0EDE2F1E0D101FA
:1032D000ED93FC93D2015296CC90D12C3F922F9239
:1032E000E1E0F0E0EC0FFD1FFF93EF9380E4882E08
:1032F000912C90E8A92EB12C22E2E22E00E026E0EB
:1033000041E8D30116966C91169714968D919C9175
:103310000E945F12082F60E870E085EE90E00E9446
:10332000370B60E870E0802F0E94280C60E870E0A6
:1033300082EE90E00E94370BF3940F900F900F9065
:103340000F9068CFED961FAEED97E1CE81E0ED9640
:103350008FAFED97DCCED2015296CC90D12C1F923C
:103360001F921F921F92912C812CB12CA12CE12C29
:10337000F301068D2BE041E26681848195810E94F4
:103380005F12082F60E870E08EEF90E00E94370B2C
:1033900060E870E0802F0E94280C60E870E08BEFFE
:1033A00090E00E94370B0F900F900F900F9000232A
:1033B00009F45ACF053009F457CF102F60E870E0B8
:1033C000812F0E94280C60E870E086EC90E00E945B
:1033D000370BD301ED91FC910480F581E02DC30101
:1033E000099520CD1F921F921F921F92912C812C24
:1033F000B12CA12CD12CC12CE12C01E023E040E028
:10340000F3016681848195810E945F12082F60E834
:1034100070E08CED90E00E94370B60E870E0802F48
:103420000E94280C60E870E089ED90E00E94370B64
:1034300060E870E089EC90E00E94370B81E0D301F6
:103440005C968C930F900F900F900F90EBCC60E8F0
:1034500070E08BEB90E00E94370BB0CF19EDE2CC1F
:10346000F701B182A08248CE3F924F925F926F9255
:103470007F928F929F92AF92BF92CF92DF92EF9204
:10348000FF920F931F93CF93DF93EC01F62E372E0D
:103490002C0182E1480E511C712C612C10E08F89A7
:1034A0008150990B681679060CF5F201C1902F0135
:1034B000D12C1F921F923F92FF9288248394912CCB
:1034C000AA24A394B12C22E0E22E00E029E041E2FC
:1034D0006E818C819D810E945F12182BFFEF6F1A05
:1034E0007F0A0F900F900F900F90D9CF812FDF910F
:1034F000CF911F910F91FF90EF90DF90CF90BF90F1
:10350000AF909F908F907F906F905F904F903F9083
:103510000895CF93DF931F92CDB7DEB78983809153
:103520001605882339F0BE016F5F7F4F8AEF94E064
:103530000E94341A8091F704882339F0BE016F5F2E
:103540007F4F8BED94E00E94341A8091D804882339
:1035500039F0BE016F5F7F4F8CEB94E00E94341A0C
:103560008091B904882339F0BE016F5F7F4F8DE9E8
:1035700094E00E94341A0F90DF91CF9108958F92BA
:103580009F92AF92BF92CF92DF92EF92FF920F93F2
:103590001F93CF93DF9300D000D0CDB7DEB77C016F
:1035A000C62ED42E590148011C821B821A82198210
:1035B0008E010F5F1F4F9E012D5F3F4F0E94700DC8
:1035C000182F882309F445C061E870E080E296E096
:1035D0000E94370B61E870E0812F0E94280C61E89F
:1035E00070E08DE196E00E94370B61E870E08BEFB0
:1035F00095E00E94370B61E870E08C2D0E94280C4A
:1036000061E870E088EF95E00E94370B61E870E0B8
:1036100088ED95E00E94370B61E870E08D2D0E94E7
:10362000280C61E870E085ED95E00E94370B812F52
:103630000F900F900F900F90DF91CF911F910F91EE
:10364000FF90EF90DF90CF90BF90AF909F908F90C2
:10365000089549815A816B817C8184019501C7015C
:103660000E94C811182FE3CF2F923F924F925F9282
:103670006F927F928F929F92AF92BF92CF92DF9282
:10368000EF92FF920F931F93CF93DF93CDB7DEB7E7
:1036900068970FB6F894DEBF0FBECDBF1B8A38E027
:1036A0003C8B3CE33D8B8A3F3FEF9307D9F416ED0B
:1036B000812F68960FB6F894DEBF0FBECDBFDF91A5
:1036C000CF911F910F91FF90EF90DF90CF90BF901F
:1036D000AF909F908F907F906F905F904F903F90B2
:1036E0002F900895222E642E362E7C01DC01169632
:1036F0000D911C911797CE01439617969C938E932C
:1037000016971A962C939E012F5F3F4F42E150E08F
:1037100060E0C7010E940314782EF7011783068327
:10372000182F8111C5CF49845A848B849C84FD81D4
:10373000FF8B3E81388F670186E5C80ED11C56018C
:103740001E8AD5018D919D915D010097D1F5BE89AD
:10375000BF5FBE8BB031A9F7F601819191916F01E6
:10376000009709F06EC07394F0E17F12F5CFF70176
:103770008681978117ED892B09F49ACF2286262D11
:1037800040E0632DC7010E948809082F14ED8823AB
:1037900009F48ECF682FC7010E94DD09009709F454
:1037A00086CFDC0114962C92602FC7010E94D313A0
:1037B000182F882309F47CCF602FC7010E94660967
:1037C00077CFDC01ED91FC910084F185E02D099526
:1037D0008111BDCFF501929182918F01DC01ED91B4
:1037E000FC910088F189E02D688D0995882309F402
:1037F000AECFF80180819181DC01ED91FC910484D0
:10380000F585E02DA401B2010995882361F0022D10
:10381000262D432D6E89C7010E94D80D182F813D9A
:1038200009F495CF45CFF80180819181DC01ED91BC
:10383000FC910684F785E02D6F8909958111E7CF0A
:1038400086CFDC01ED91FC910084F185E02D099596
:10385000811189CFF601929182918F01DC01ED9166
:10386000FC910088F189E02D688D099581110DC0CA
:10387000022D262D432D672DC7010E94D80D182F2C
:10388000877F813D09F014CF6ECFF801808191814F
:10389000DC01ED91FC910484F585E02DA401B201D9
:1038A0000995811160CFF80180819181DC01ED9152
:1038B000FC910684F785E02D6F8909958823C1F274
:1038C00052CFEF92FF920F931F93CF930E94BA0EA5
:1038D0008091F903813041F058F0823009F460C0E2
:1038E000833069F0C0E022C083E180934A04FACFBC
:1038F00080914A04807F8031A9F381E1F6CFC1E055
:1039000080914A04807F803189F40E94120A6853B2
:103910007F4F8F4F9F4F6093F5037093F603809313
:10392000F7039093F80380E280934A048FE6E82E31
:1039300085E0F82E8701D8018D919D918D0100972A
:1039400039F0DC01ED91FC910680F781E02D0995BD
:10395000B5E00F381B0779F780914A04803409F4E9
:103960006BC000F5803209F451C0803309F45EC0A9
:103970008131F9F410928F05F701819191917F01C6
:10398000009739F0DC01ED91FC910480F581E02D88
:1039900009950E151F0581F782E180934A0409C03D
:1039A000C0E0AECF813509F471C048F4803509F428
:1039B00056C0CF911F910F91FF90EF9008958038DE
:1039C00009F477C0803AA9F760E870E088E496E0EF
:1039D0000E94370B60E870E08091F4030E94280C8D
:1039E00060E870E085E496E00E94370B0E94120ABE
:1039F00068537F4F8F4F9F4F6093F5037093F6038B
:103A00008093F7039093F80380E2C7CF0E94120AD5
:103A10000091F5031091F6032091F7033091F8031C
:103A2000601B710B820B930B97FDC3CF61E088EE97
:103A30000E94EC0C80E4B1CF88EE0E94FF0C80FD68
:103A4000B8CF60E488EC0E94EC0C88ED0E94FF0C7B
:103A5000682F686088ED0E94EC0C80E59ECF88ECB2
:103A60000E94FF0C86FFA5CF81E580934A040E9447
:103A7000120A6C507E4F8F4F9F4F6093F5037093E7
:103A8000F6038093F7039093F80393CF0E94120AF2
:103A90000091F5031091F6032091F7033091F8039C
:103AA000601B710B820B930B97FD83CF80E8809393
:103AB0004A042C2F40E060E089E195E00E94341B2D
:103AC000882339F0823D09F474CF8093F40380EAAF
:103AD00064CF80E962CFCF92DF92EF92FF921F9383
:103AE000CF93DF93EC01162F7A01FA018081918147
:103AF000A281B3818130F3E09F07F1E0AF07B10508
:103B0000C9F170F48115E1E09E07AE07B10509F433
:103B100050C081309140A140B10561F180E041C0C9
:103B2000833021E0920720E1A207B10529F083301C
:103B30009340A041B10591F7412F64E1CE010E946D
:103B4000A514412F60E1CE010E94A51464E170E04C
:103B500080E090E00E948D0B6A85F7012181269517
:103B600021706770412F8A819B810E94341B1092C3
:103B70009602D4CF809196028111D0CF412F61E17E
:103B8000CE010E94A514412F60E1CE010E94A51430
:103B9000412F64E0CE010E94F91481E080939602E7
:103BA00081EBDF91CF911F91FF90EF90DF90CF904D
:103BB0000895462F61E1CE010E94A514412F60E1D6
:103BC000CE010E94A514109296028A858770177004
:103BD000880F880F880F182B09F4A0CFEA80FB808C
:103BE0006701F6E5CF0ED11CD0E0C0E0D6018D9183
:103BF0009D916D010097C1F0DC01ED91FC91008475
:103C0000F185E02D099518130FC0AB96CC0FDD1F81
:103C1000CE0DDF1D88819981DC01ED91FC9104803E
:103C2000F581E02D09957ACF2196C031D105F1F6C5
:103C300075CFCF92DF92EF92FF920F931F93CF93A6
:103C4000DF93CDB7DEB72E970FB6F894DEBF0FBE69
:103C5000CDBFFC012089211111C010E0812F2E96CB
:103C60000FB6F894DEBF0FBECDBFDF91CF911F918D
:103C70000F91FF90EF90DF90CF9008957C010E940C
:103C8000120AF7010485158526853785601B710B9F
:103C9000820B930B97FDE1CF81E090E09E878D87AB
:103CA0008E010F5F1F4F9E01235F3F4F41E06285F2
:103CB000828193810E94BF1A182F811121C082E056
:103CC000D82E01E089818D2139F119861A861B864B
:103CD0001C86AE01475F5F4F602FC7010E94CE1464
:103CE000C82E811119C0AE01475F5F4F602FC70119
:103CF0000E946B1D813B19F0882371F0C82E1C2D8A
:103D00000E94120A6C597F4F8F4F9F4FF7016487B3
:103D1000758786879787A2CFDD0C0F5F083091F6F5
:103D200001E0F7018385801758F319861A861B86F0
:103D30001C86AE01475F5F4F602FC7010E94CE1403
:103D4000D82E811117C089859A858770917081302E
:103D5000914081F48B859C8581609C878B87AE0127
:103D6000475F5F4F602FC7010E946B1D813B29F0A9
:103D7000811102C00F5FD5CFD82E1D2DC1CF0F935B
:103D80001F93CF93DF938091EE039091ED03892BE6
:103D900080938E029091EC03992389F0892B809374
:103DA0008E02EFE8F2E026E932E080E09191911195
:103DB0008F5F2E173F07D1F781111092EC03E0912E
:103DC000EA03F091EB033097B1F10280F381E02D2B
:103DD0008EE892E009958091E90382FF2CC080FF74
:103DE00004C08AEC95E00E948A03D0E0C0E004ECB5
:103DF00015E08091E90380FF0EC0FE01E257FD4F00
:103E000080811F928F931F930F930E9423040F9022
:103E10000F900F900F902196C830D10551F78091E7
:103E2000E90380FF08C082EC95E0DF91CF911F91FC
:103E30000F910C948A03DF91CF911F910F910895F8
:103E40001092ED03EEE8F2E01182128213821482E6
:103E50001582168217820C94BF1ECF93DF93209198
:103E6000E7023091E8022817390701F19093E80240
:103E70008093E702E091EA03F091EB033097B1F011
:103E8000EC010084F185E02D09958091E9038570AE
:103E9000853061F4DF93CF9382EB94E09F938F930F
:103EA0000E9423040F900F900F900F90DF91CF91FD
:103EB0000895CF93DF932091E5023091E602281711
:103EC000390701F19093E6028093E502E091EA035D
:103ED000F091EB033097B1F0EC010680F781E02D13
:103EE00009958091E9038570853061F4DF93CF9364
:103EF00084EA94E09F938F930E9423040F900F9085
:103F00000F900F90DF91CF910895FF920F931F9321
:103F1000CF93DF9300D000D01F92CDB7DEB7498397
:103F2000952F5A836B837C838D832C813D8181E027
:103F30002115310531F05F3F19F481E04F3F09F061
:103F400080E080FD49C081E0232B31F09F3F19F4D0
:103F500081E04F3F09F080E02B8180FD54C0692F44
:103F600070E050E0CB01E4E0880F991FEA95E1F79B
:103F700087519D4FDC01A40FB51F222309F437C0E0
:103F80001C9280E090E1899FF0011124E60FF71F59
:103F900034E0EE0FFF1F3A95E1F7E40FF51FEE5303
:103FA000FB4FE49180E48E0F803218F5E05CFF0B4C
:103FB000EE0FFF1FEE53FA4F85919491FC011E2FD7
:103FC0008F2F82958F70823008F4CAC08E3021F412
:103FD000E11102C02111BAC10F900F900F900F9004
:103FE0000F90DF91CF911F910F91FF9008958C91C9
:103FF000C9CFEF3B58F4E83A30F5E53AB8F4E4308D
:1040000080F4E13081F0F0E0E0E0D9CFE83E38F430
:10401000E03E38F4EF3BB9F7E0E0F0EED0CFE03F20
:1040200090F3F0E0CCCFE1E0F0E0C9CFE53A29F041
:10403000E63A31F4E2E8F0E4C2CFE1E8F0E4BFCFE1
:10404000E3E8F0E4BCCFE83A09F445C0E93A09F402
:1040500045C0EA3A09F445C0EB3A09F445C0EC3AE8
:1040600009F445C0ED3A09F445C0EE3A09F445C0FB
:10407000EF3A09F445C0E13B09F445C0E03B09F4DF
:1040800045C0E23B09F445C0E33B09F445C0E43BCD
:1040900009F445C0E53B09F445C0E63B09F445C0D9
:1040A000E73B09F445C0E83B09F445C0E93B09F4A6
:1040B00045C0EA3B09F445C0EB3B09F445C0EC3B85
:1040C00009F445C0ED3B09F445C0EE3B09F045C09D
:1040D000E0E7F4E474CFE2EEF4E471CFE9EEF4E467
:1040E0006ECFEAEEF4E46BCFE5EBF4E468CFE6EBF9
:1040F000F4E465CFE3EBF4E462CFE4EBF4E45FCF08
:10410000E7EBF4E45CCFECECF4E459CFEDECF4E451
:1041100056CFE3E8F5E453CFEAE8F5E450CFE2E91F
:10412000F5E44DCFE4E9F5E44ACFE1E2F6E447CF28
:10413000E3E2F6E444CFE4E2F6E441CFE5E2F6E47C
:104140003ECFE6E2F6E43BCFE7E2F6E438CFEAE240
:10415000F6E435CFEFE6F4E432CFE0E0F4E42FCF3D
:104160008F2F8F70F82E8F2F807F19F0F29480EFB1
:10417000F822222309F4F9C0FF2039F08091ED03E1
:104180008F298093ED030E94BF1E112309F424CFD1
:104190008EE7810F833070F5123831F1133839F51D
:1041A00011E003E50E948B04812309F015CF802FD5
:1041B0000E9472040E94BF1E9FEF21EE84E0915086
:1041C00020408040E1F700C00000802F0E9466047C
:1041D0000F900F900F900F900F90DF91CF911F9144
:1041E0000F91FF900C94BF1E12E009E3DBCF14E0A7
:1041F00007E4D8CF8CEF810F813A20F4812F0E9401
:104200007204E6CF80E2810F883068F4177021E0F5
:1042100030E001C0220F1A95EAF78091EE03822B5D
:104220008093EE03D5CF8BE5810F8330B0F481E826
:1042300090E0153A31F082E890E0163A11F083E808
:1042400090E00F900F900F900F900F90DF91CF9113
:104250001F910F91FF900C94591F88E5810F8731B2
:1042600008F071C082EE90E0183A09F460C089EE5F
:1042700090E0193A09F45BC08AEE90E01A3A09F42A
:1042800056C085EB90E01B3A09F451C086EB90E0F4
:104290001C3A09F44CC083EB90E01D3A09F447C086
:1042A00084EB90E01E3A09F442C087EB90E01F3A9D
:1042B000F1F18CEC90E0113BD1F18DEC90E0103BF2
:1042C000B1F183E891E0123B91F18AE891E0133B70
:1042D00071F182E991E0143B51F184E991E0153BE1
:1042E00031F181E292E0163B11F183E292E0173B5B
:1042F000F1F084E292E0183BD1F085E292E0193BC4
:10430000B1F086E292E01A3B91F087E292E01B3B2B
:1043100071F08AE292E01C3B51F08FE690E01D3B89
:1043200031F080E790E01E3B11F090E080E00F90CC
:104330000F900F900F900F90DF91CF911F910F91E1
:10434000FF900C942D1F1F3B09F046CE1092EE03F8
:104350000E94201F9FEF20E782E091502040804084
:10436000E1F700C000000E94B604112309F18EE7B6
:10437000810F833070F5123831F1133839F511E0BF
:1043800003E50E948B04812399F0802F0E94720420
:104390000E94BF1E9FEF21EE84E09150204080409C
:1043A000E1F700C00000802F0E9466040E94BF1E3B
:1043B000FF2009F411CE8F2D80959091ED03892374
:1043C0008093ED0305CF12E009E3DBCF14E007E4AF
:1043D000D8CF8CEF810F813A10F4812FE5CF80E2A6
:1043E000810F883070F4177021E030E001C0220F97
:1043F0001A95EAF720959091EE0329232093EE0376
:10440000D5CF8BE5810F833028F490E080E00E94C7
:10441000591FCECF185A173158F690E080E00E940D
:104420002D1FC6CFEF92FF920F931F93CF93DF9371
:104430002091E4022430B1F521E02093E90021E845
:10444000215021F03091E80035FF33C02091E80081
:1044500025FF28C0C92FD82F0E943405811114C010
:104460000D2F1C2F88E0E82EF12C8091E80085FDAF
:1044700027C08091E8008E778093E8000E94B40501
:104480000E943405882389F38091E8008E77809319
:10449000E80088E0ED2FFC2FA1EDB2E001900D9235
:1044A0008A95E1F7DF91CF911F910F91FF90EF90E7
:1044B0000895EFE3F1E03197F1F700C00000C0CFBD
:1044C000F80181918F018093F100F1E0EF1AF1087A
:1044D00061F6DACF8F929F92AF92BF92DF92EF9206
:1044E000FF920F931F93CF93DF937C01CB01D22ECA
:1044F000DB01ED91FC910084F185E02D09951F927F
:104500008F938EEA92E09F938F930E942304E80199
:1045100048018D0C911C0F900F900F900F9088EA1E
:10452000A82E82E0B82EC815D90561F089911F9296
:104530008F93BF92AF920E9423040F900F900F9021
:104540000F90F1CF85EA92E09F938F930E9423040E
:104550000F900F90B8E08AE992E0DB1206C0F801F4
:1045600082818130A1F480E892E09F938F930E9432
:1045700023040F900F90DF91CF911F910F91FF9027
:10458000EF90DF90BF90AF909F908F900895D701EC
:10459000129688E001900D928A95E1F70E94120A26
:1045A000D7011B967C936E931A97E5CF2F923F927B
:1045B0005F926F927F928F929F92AF92BF92CF92B3
:1045C000DF92EF92FF920F931F93CF93DF9300D070
:1045D00000D000D0CDB7DEB77C012DB73EB73E830B
:1045E0002D83DC015C968C91811121C0512C852D8D
:1045F0002D813E810FB6F8943EBF0FBE2DBF26968B
:104600000FB6F894DEBF0FBECDBFDF91CF911F91E3
:104610000F91FF90EF90DF90CF90BF90AF909F9061
:104620008F907F906F905F903F902F9008950E94A1
:10463000120AF701008D118D228D338D601B710BD5
:10464000820B930B97FDD2CF6701B12CA12C512C7B
:10465000D70157968C918150990BA816B9060CF08A
:1046600009C1EDB7FEB7FC83EB8361E870E081E739
:1046700092E00E94370B61E870E0C5010E94070CD0
:1046800061E870E08EE692E00E94370B61E870E02E
:104690008BE392E00E94370B3501FFEF6F1A7F0A20
:1046A00061E870E0D6011A968C910E94280C61E8AE
:1046B00070E088E392E00E94370B61E870E081E0EF
:1046C00092E00E94370B61E870E0F60183850E945A
:1046D000280C61E870E08EEF91E00E94370BD60164
:1046E0001B968C9190E08134910508F053C09A8319
:1046F000898389819A812DB73EB7281B390B0FB664
:10470000F8943EBF0FBE2DBF8DB79EB701964C01EA
:104710008C019E012F5F3F4FD6011A964C91F701F5
:104720006681848195810E94BF1A582E811137C0FD
:1047300029813A8123303105B0F1D70150968D910E
:104740009C91009749F0DC01ED91FC910190F08182
:10475000E02D40E0B701099589819A8110E0892B0D
:1047600009F47CC029813A81812F90E08217930758
:1047700008F06CC0880D991D60E870E0DC018C9138
:104780000E94280C60E870E089EA91E00E94370BF3
:104790001F5FE8CFE0E4F0E0FA83E983AACFB4E05A
:1047A0008B1709F45BC061E870E08CEE91E00E9429
:1047B000370B61E870E0852D0E94280C61E870E0FD
:1047C00089EE91E00E94370B511048C089819A818F
:1047D000892B09F443C060E870E088EC91E00E9406
:1047E000370B29803A800CE010E0C101002E02C096
:1047F000969587950A94E2F7982F9F7080E3890F2A
:104800008A3310F087E3890F60E870E00E94310B73
:10481000045011090C3FEFEF1E0739F760E870E014
:1048200085EC91E00E94370B60E870E08EEA91E041
:104830000E94370B60E870E0C5010E94070C60E839
:1048400070E08BEA91E00E94370B86CF232B31F08A
:1048500060E870E086EA91E00E94370BEB81FC8112
:104860000FB6F894FEBF0FBEEDBFF3E0CF0ED11C24
:104870005301EECE0E94120AD7015D962C91620F71
:10488000711D811D911DF701608F718F828F938F34
:10489000AECECF931092FD031092FC0388EE93E00E
:1048A000A0E0B0E08093FE039093FF03A093000488
:1048B000B093010487E591E09093FB038093FA03A2
:1048C0008FEF9FEF90930704809306048FE791E0AA
:1048D00090931A05809319051092210581E0809329
:1048E0002205109223058BE195E09093200580939B
:1048F0001F0510921B0588E080931C058CE38093B4
:104900001D0510921E05E9E1F5E0C1E08BE195E09F
:104910001586C687178694878387359625E0E43603
:10492000F207B1F710928F0581E180934A048AEF74
:1049300094E00E942C048BED94E00E942C048CEBFC
:1049400094E00E942C048DE994E00E942C0489E8F4
:1049500091E09093920480939104909386048093C5
:10496000850490937A048093790490936E048093E5
:104970006D0489E691E090935D0480935C0489E185
:1049800095E090935F0480935E0410926C04109203
:10499000600488E0809361049CE390936204C09378
:1049A00063048093640484E0809365041092660439
:1049B00010926704109268041092690410926A04BD
:1049C00010926B04AFE6B5E0FD0190E080E021912C
:1049D0003191232B09F044C0880F991FFC01E15944
:1049E000FA4F8CE594E09183808389E691E090937F
:1049F0004C0480934B0489E195E090934E0480939E
:104A00004D0410925B0410924F0488E08093500490
:104A10009CE39093510491E090935204809353044B
:104A200084E080935404109255041092560410921E
:104A30005704109258041092590410925A0490E0AE
:104A400080E02D913D91232B89F4880F991FFC0163
:104A5000E159FA4F8BE494E091838083CF910895DC
:104A600001968031910509F0B2CFBFCF0196803118
:104A7000910539F7F3CF1F920F920FB60F921124C1
:104A80008F939F93AF93BF938091F303811113C0D2
:104A90008091EF039091F003A091F103B091F203A4
:104AA0004196A11DB11D8093EF039093F003A09355
:104AB000F103B093F203BF91AF919F918F910F904B
:104AC0000FBE0F901F9018951F920F920FB60F9266
:104AD00011242F933F934F935F936F937F938F9303
:104AE0009F93AF93BF93CF93DF93EF93FF93809107
:104AF000E10082FF09C08091E20082FF05C0809141
:104B0000E1008B7F8093E1008091DA0080FF1FC07D
:104B10008091D80080FF1BC08091DA008E7F809347
:104B2000DA008091D90080FF41C180E189BD82E136
:104B300089BD09B400FEFDCF81E08093E40280913D
:104B4000CD02811104C00E9497040E9483088091C5
:104B5000E10080FF4FC08091E20080FF4BC0809158
:104B6000E2008E7F8093E2008091E200806180937A
:104B7000E2008091D80080628093D80019BC85E063
:104B80008093E4028091E90380FF08C08DE993E0FF
:104B90009F938F930E9423040F900F908091CE02D9
:104BA000882341F11092EE030E94201F62E088ECFE
:104BB0000E94EC0C88ED0E94FF0C682F677F88ED47
:104BC0000E94EC0C8091DA02811114C08091E903FB
:104BD00080FF08C089E993E09F938F930E9423048C
:104BE0000F900F9061E088E60E94EC0C60E188E78E
:104BF0000E94EC0C8091E10084FF83C08091E20070
:104C000084FF7FC080E189BD82E189BD09B400FED7
:104C1000FDCF8091D8008F7D8093D8008091E100F6
:104C20008F7E8093E1008091E2008F7E8093E2008E
:104C30008091E20081608093E2008091DB02882312
:104C400009F4BAC084E08093E4028091E90380FF14
:104C500008C085EA93E09F938F930E9423040F90EE
:104C60000F908091CE02882309F44BC01092EE037E
:104C70000E94201F8091DA02811129C08091E903EE
:104C800080FF08C081EA93E09F938F930E942304E2
:104C90000F900F9060E088E70E94EC0C88E60E947D
:104CA000FF0C8823D9F3CFE6D5E08991999100973D
:104CB00039F0DC01ED91FC910480F581E02D09953E
:104CC000B5E0CF38DB0789F780E180934A0468E0DC
:104CD00088EE0E94EC0C88EE0E94FF0C83FDFBCF57
:104CE00060E488EC0E94EC0C88ED0E94FF0C682FB9
:104CF000686088ED0E94EC0C88EC0E94FF0C86FF37
:104D0000FBCF8091E10083FF3EC08091E20083FFF2
:104D10003AC08091E100877F8093E10082E0809338
:104D2000E4021092DB028091E1008E7F8093E1002B
:104D30008091E2008E7F8093E2008091E2008061AA
:104D40008093E20042E060E080E00E94820581E022
:104D5000809310011092CF021092D00288E0E1ED12
:104D6000F2E0DF011D928A95E9F710928F0210920E
:104D7000900210929102109292021092930210925D
:104D8000940210929502FF91EF91DF91CF91BF9124
:104D9000AF919F918F917F916F915F914F913F91D3
:104DA0002F910F900FBE0F901F90189519BC109265
:104DB000E4021092CD02CBCE8091E30087FD02C0C9
:104DC00081E041CF83E03FCFCF93DF93CDB7DEB714
:104DD0002A970FB6F894DEBF0FBECDBF84B7877F8A
:104DE00084BF0FB6F894A895809160008861809385
:104DF0006000109260000FBE80E890E00FB6F8945B
:104E000080936100909361000FBE8DE29BE09093D0
:104E10008D0180938C0186E091E09093EB03809369
:104E2000EA0384E793E00E948A030E9497040E94A9
:104E30008308789482E084BD93E095BD9AEF97BD96
:104E400080936E008091E90381608093E903269A44
:104E50000E94C60C219A229A2398209A80E58CBD44
:104E600081E08DBD259868E188E80E94EC0C60E245
:104E700088E70E94EC0C60E088E70E94EC0C10E0F0
:104E800000E088E60E94FF0C0F5F1F4F80FF1CC0F0
:104E900061EC88ED0E94EC0C60E280ED0E94EC0C6D
:104EA00064E088EE0E94EC0C88EE0E94FF0C82FF0A
:104EB000FBCF0E94BA0E60E288EC0E94EC0C61E02D
:104EC00080E80E94EC0C03C00F3F1007D1F681E987
:104ED00094E090930B0580930A0585E894E0909305
:104EE000EC048093EB0489E794E09093CD048093E5
:104EF000CC048DE694E09093AE048093AD040EE074
:104F000013E068E0E62E63E0F62E8091E402843040
:104F100009F00DC10E941E0A882309F408C182E627
:104F200093E00E948A038091E90380FF08C086E134
:104F300093E09F938F930E9423040F900F9081E042
:104F40008093CE0284E593E00E948A0349E2442ED6
:104F500043E0542E5EE1652E53E0752E8091E4020D
:104F6000853009F41CC160919B0470919C044091B0
:104F70008F04509190042091830430918404809197
:104F8000770490917804E091A002F091A1026E174D
:104F90007F07B1F4E0919E02F0919F024E175F07E8
:104FA00079F4E0919C02F0919D02E217F30741F43D
:104FB000E0919A02F0919B028E179F0709F45FC05F
:104FC0007093A1026093A00250939F0240939E02AF
:104FD00030939D0220939C0290939B0280939A02AF
:104FE00088E0E2EAF2E0DF011D928A95E9F720917C
:104FF00093043091940440919504509196046091EB
:105000009704709198048091990490919A040E9459
:10501000170F2091870430918804409189045091A2
:105020008A0460918B0470918C0480918D0490911E
:105030008E040E94170F20917B0430917C044091D4
:105040007D0450917E0460917F0470918004809172
:105050008104909182040E94170F20916F04309177
:1050600070044091710450917204609173047091C6
:10507000740480917504909176040E94170F0E9429
:10508000310A8C010E94611C2FB7F8948091EF03C4
:105090009091F003A091F103B091F2032FBF801B18
:1050A000910B8536910560F09F938F938AE393E08F
:1050B0009F938F930E9423040F900F900F900F9057
:1050C00080914A0490919902981729F1809399024E
:1050D0001F928F935F924F920E9423040F900F9024
:1050E0000F900F90809199028039A9F48091F90373
:1050F000823009F0BDC084E191E09F938F937F924D
:105100006F920E9423040E948B040E94891A0F90C0
:105110000F900F900F902BEAE22E22E0F22E30E259
:10512000832E99249A94312C10E000E0AFC00E94A5
:10513000B4050E94611C80914A04909198029817CE
:1051400009F4E3CE809398029091E90390FF0AC09E
:105150001F928F931F930F930E9423040F900F9021
:105160000F900F9080919802803909F0CECE8091F7
:10517000E90380FFCACE8091F903823069F482E1AD
:1051800091E09F938F93FF92EF920E9423040F90E0
:105190000F900F900F90B9CE87E191E0F2CF809100
:1051A000E90380FF08C08AE193E09F938F930E94F8
:1051B00023040F900F908091E402843021F110922B
:1051C000F30388E190E020E40FB6F894A89580936B
:1051D00060000FBE2093600083B7817F846083BF2F
:1051E00083B7816083BF7894889583B78E7F83BFB0
:1051F0000FB6F894A8958091600088618093600054
:10520000109260000FBE8091DA02882309F4A6CEC6
:1052100088EC0E94FF0C81FF1AC062E088EC0E94BB
:10522000EC0C80E189BD82E189BD09B400FEFDCFAF
:105230008091D8008F7D8093D8008091E0008260BB
:105240008093E0008091E00081FDFCCF87CE64E098
:1052500088EE0E94EC0C88EE0E94FF0C82FFFBCFD0
:1052600088EF0E94FF0C807C803409F077CED9CF84
:1052700089E191E042CFB8E08B16910408F054CF59
:105280000091A202002309F44FCF10E0E4EAF2E01B
:105290008191843080F0982F92959F7039120BC0C5
:1052A0008F7021E030E002C0220F331F8A95E2F7B1
:1052B000C901022B192B32E0EA3AF30749F7D7016B
:1052C000AD90BC90A016B10671F1212CCC24C394F2
:1052D000D12CA026B126C5018C219D21892BE9F076
:1052E0002E823F8221E0C8018C219D21892B09F467
:1052F00020E028870E94310A8160782F9A87898769
:105300004E815F8168858A850E94851FF7018081B3
:1053100091818C259D25918380832394CC0CDD1C69
:10532000F0E12F12D8CF339420E1820E911C32E0AD
:10533000E30EF11C80E138129ECF8FEF89838A83C0
:105340001B820E94310A8160782F9D838C83498162
:105350005A816B818D810E94851F0E948B049091E0
:10536000AA028917C9F00E948B048093AA02909127
:10537000E9039570953061F41F928F93A9E4B3E02F
:10538000BF93AF930E9423040F900F900F900F9044
:105390008091AA020E94891A2091E4003091E500D0
:1053A0008091CB029091CC022817390739F1809176
:1053B000E4009091E5009093CC028093CB020E9490
:1053C0001E0A8823D9F08091E4028430B9F48091D8
:1053D000E9008F709091EC0090FF13C090E8892B4A
:1053E00093E09093E9009091EB0090FF04C09091BE
:1053F000EE0097FD24C08F708093E9000E94B405F1
:10540000ADCD90E0ECCFE0910101F0910201E90F08
:10541000F11D20819F5F309105019323909304013A
:105420002093F1009091E80095FD09C09091E8006B
:1054300090FF05C09091E8009E779093E8009091CE
:10544000040120910301291721F02091E80025FD96
:10545000DACF2091F3009091F200322F292F232BE5
:1054600051F29091E80090FFC6CF9091E80095FD31
:1054700006C09091E8009E779093E800BCCF109210
:10548000F100F3CF78941F920F920FB60F92112470
:105490008F939F93AF93BF938091EF039091F0030D
:1054A000A091F103B091F2030196A11DB11D80936B
:1054B000EF039093F003A093F103B093F203BF9135
:1054C000AF919F918F910F900FBE0F901F901895E5
:1054D0000E94D92A08F481E008950E94052B88F0E3
:1054E0009F5798F0B92F9927B751B0F0E1F0660FA8
:1054F000771F881F991F1AF0BA95C9F714C0B130E9
:1055000091F00E941F2BB1E008950C941F2B672F80
:10551000782F8827B85F39F0B93FCCF38695779517
:105520006795B395D9F73EF4909580957095619500
:105530007F4F8F4F9F4F0895E89409C097FB3EF42B
:1055400090958095709561957F4F8F4F9F4F9923D0
:10555000A9F0F92F96E9BB279395F695879577954E
:105560006795B795F111F8CFFAF4BB0F11F460FF0E
:105570001BC06F5F7F4F8F4F9F4F16C0882311F066
:1055800096E911C0772321F09EE8872F762F05C07A
:10559000662371F096E8862F70E060E02AF09A9515
:1055A000660F771F881FDAF7880F9695879597F90A
:1055B0000895990F0008550FAA0BE0E8FEEF1616A4
:1055C0001706E807F907C0F012161306E407F507F7
:1055D00098F0621B730B840B950B39F40A2661F06B
:1055E000232B242B252B21F408950A2609F4A1400E
:1055F000A6958FEF811D811D089557FD9058440F8A
:10560000551F59F05F3F71F04795880F97FB991F21
:1056100061F09F3F79F087950895121613061406DE
:10562000551FF2CF4695F1DF08C01616170618066B
:10563000991FF1CF86957105610508940895E89446
:10564000BB2766277727CB0197F908950E94D92AAF
:1056500008F48FEF08950E943E2B0C94AF2B0E940C
:10566000A12B38F00E94A82B20F0952311F00C9468
:10567000982B0C949E2B11240C94202B0E94FD2A15
:1056800070F3959FC1F3950F50E0551F629FF00195
:10569000729FBB27F00DB11D639FAA27F00DB11DAE
:1056A000AA1F649F6627B00DA11D661F829F222737
:1056B000B00DA11D621F739FB00DA11D621F839FBE
:1056C000A00D611D221F749F3327A00D611D231F94
:1056D000849F600D211D822F762F6A2F11249F57E2
:1056E00050409AF0F1F088234AF0EE0FFF1FBB1FE5
:1056F000661F771F881F91505040A9F79E3F5105A4
:1057000080F00C94982B0C94202B5F3FE4F3983E90
:10571000D4F3869577956795B795F795E7959F5F4D
:10572000C1F7FE2B880F911D9695879597F90895DF
:1057300097F99F6780E870E060E008959FEF80EC44
:10574000089500240A9416161706180609060895E7
:1057500000240A9412161306140605060895092E4D
:105760000394000C11F4882352F0BB0F40F4BF2BBC
:1057700011F460FF04C06F5F7F4F8F4F9F4F0895FC
:10578000EE0FFF1F0590F491E02D0994F894FFCFE0
:10579000058E010000FFE7081222E608E408E5088C
:1057A00001FF660066756C6C006C6F77000000008E
:1057B00000860F00000000A71000000000060C008B
:1057C000000000D716C611A90CD622A60CC511C31D
:1057D00011A10C9C0C910C0B0F080F4A0CFEFF0042
:1057E00000870C00000000F60BDC0BFD0BFC0B032C
:1057F0000C000C000C000000007D15C611EA081911
:105800001E11092215C3110C09100A00000000DD49
:0C5810000988096609000000006A2200F7
:00000001FF
